:1000000010C028C028C087C025C024C023C022C07B
:1000100021C020C01FC01EC01DC01CC01BC01AC0F4
:1000200019C011241FBECFEDCDBF10E0A0E6B0E097
:10003000E4E7F5E003C0C89531960D92A836B10704
:10004000D1F710E0A8E6B0E001C01D92AC37B107CF
:10005000E1F7C1C0D5CF1F920F920FB60F921124B6
:100060002F933F934F935F938F939F93AF93BF9340
:100070008CB59DB5282F392F44275527C89B09C01B
:1000800020937700309378004093790050937A0062
:1000900035C08091770090917800A0917900B0915F
:1000A0007A00281B390B4A0B5B0B20936E003093B0
:1000B0006F00409370005093710080916E0090919A
:1000C0006F00A0917000B0917100B7FF14C08091D3
:1000D0006E0090916F00A0917000B09171008050FF
:1000E0009040AF4FBF4F80936E0090936F00A093EE
:1000F0007000B093710081E080936900BF91AF916F
:100100009F918F915F914F913F912F910F900FBED3
:100110000F901F9018951F920F920FB60F921124F7
:100120002F933F934F935F938F939F93AF93BF937F
:100130008CB59DB5282F392F44275527B09B09C072
:1001400020936A0030936B0040936C0050936D00D5
:1001500035C080916A0090916B00A0916C00B091C5
:100160006D00281B390B4A0B5B0B209373003093F7
:1001700074004093750050937600809173009091C5
:100180007400A0917500B0917600B7FF14C0809103
:10019000730090917400A0917500B091760080502A
:1001A0009040AF4FBF4F8093730090937400A09323
:1001B0007500B093760081E080937B00BF91AF9192
:1001C0009F918F915F914F913F912F910F900FBE13
:1001D0000F901F9018958F929F92AF92BF92CF92DF
:1001E000DF92EF92FF920F931F93CF93DF9380E8FC
:1001F00086BD16BC80E090E00000019620E28030D1
:100200009207D1F7A0E0B0E097D1EF5FFF4FA9F4DC
:10021000E0E6F0E020E030E043E050E0E199FECF9E
:1002200081919191B32FA22F082E192E8AD141507E
:1002300050402E5F3F4F57FFF1CF88E28BBB81E0EC
:1002400082BB80BD80E38BBF83EA80BF83E083BF36
:1002500080E886BF8CBF8FEF9FEF9BBD8ABD1FBC20
:1002600089E08EBD84E087BB80ED8ABB1092690077
:1002700010927B007894A0E0B0E05ED1CE2EDF2E0D
:10028000A2E0B0E059D18E2E9F2EA4E0B0E054D170
:10029000CE2FDF2FA6E0B0E04FD1AE2EBF2E8BB316
:1002A00080658BBB809169008823E1F1E0906E004E
:1002B000F0906F0000917000109171008C2D9D2DB9
:1002C000AA27BB27E81AF90A0A0B1B0B17FF04C061
:1002D000EE24FF24002711272FEF30E040E050E00C
:1002E000912F802F7F2D6E2DCAD0392D282D2C19BE
:1002F0003D0944275527DED02F3F310541055105E3
:1003000011F00CF0B2C026BF1092690025573040A2
:1003100040405040273131054105510510F4DC9A29
:1003200001C0DC9880917B008823E1F1E0907300AC
:10033000F090740000917500109176008C2F9D2F25
:10034000AA27BB27E81AF90A0A0B1B0B17FF04C0E0
:10035000EE24FF24002711272FEF30E040E050E08B
:10036000912F802F7F2D6E2D8AD03B2D2A2D2C1B77
:100370003D0B442755279ED02F3F310541055105A0
:1003800011F00CF077C02CBF10927B002557304045
:1003900040405040273131054105510510F4DE9AA7
:1003A00001C0DE98CB992EC080916800882351F55A
:1003B00080916E0090916F00A0917000B0917100DB
:1003C000C82ED92E8091730090917400A091750071
:1003D000B0917600D92FC82F8CB39927B92FA82FA9
:1003E000A270B07081FDF8CF0C2C1D2CAAD0E19921
:1003F000FECFA4E0B0E00C2E1D2EA3D081E08093B0
:10040000680002C010926800CD992CC080917200E3
:10041000882341F580916E0090916F00A09170004B
:10042000B0917100882E992E809173009091740084
:10043000A0917500B0917600A82EB92EE199FECF5B
:10044000A2E0B0E0082C192C7CD0E199FECFA6E008
:10045000B0E00A2C1B2C75D0CD9BFECF81E08093A1
:10046000720020CF109272001DCF8FEF86BF1092C6
:10047000690057CF8FEF8CBF10927B0092CFFF2780
:10048000EE27BB27AA2760FF04C0A20FB31FE41FFB
:10049000F51F220F331F441F551F9695879577959B
:1004A000679589F70097760771F79F2F8E2F7B2F1F
:1004B0006A2F089597FB092E05260ED057FD04D00C
:1004C00014D00AD0001C38F45095409530952195F1
:1004D0003F4F4F4F5F4F0895F6F790958095709579
:1004E00061957F4F8F4F9F4F0895A1E21A2EAA1B4F
:1004F000BB1BEA2FFB2F0DC0AA1FBB1FEE1FFF1F48
:10050000A217B307E407F50720F0A21BB30BE40B17
:10051000F50B661F771F881F991F1A9469F760955E
:10052000709580959095262F372F482F592F6A2F39
:100530007B2F8E2F9F2F089509D0E02D07D0F02D0F
:1005400008950CD0012C0AD011240895E199FECF12
:10055000BFBBAEBBE09A11960DB20895E199FECFF4
:10056000BFBBAEBB0DBA11960FB6F894E29AE19AF2
:040570000FBE08951D
:08057400FF190040FF190040CF
:00000001FF
